:10136200EA6000D20000010001400160018001A09A
:1013720001C001E002000300039603B603D603F4A2
:10138200040005000518053005480560057805903C
:1013920005A805C0060006140628063C066E068C43
:1013A20000FF013F015F017F019F01BF01DF01FFDC
:1013B20002FF039503B503D503F303FF04FF0517EB
:1013C200052F0547055F0577058F05A705BF05FFB3
:1013D20006130627063B066F068B06FF0FAA0FA50C
:1013E2000F9F0F9A0F940F8D0F870F800F780F7139
:1013F2000F680F600F570F4E0F450F3B0F300F2531
:101402000F1A0F0E0F020EF50EE80EDB0ECC0EBEFB
:101412000EAE0E9F0E8E0E7D0E6C0E5A0E470E34C1
:101422000E200E0C0DF70DE20DCB0DB50D9D0D85A9
:101432000D6D0D540D3A0D200D050CE90CCE0CB1BD
:101442000C940C760C580C3A0C1B0BFB0BDB0BBBF5
:101452000B9A0B790B570B350B130AF10ACE0AAB19
:101462000A870A640A400A1C09F809D409B0098CDF
:1014720009670943091F08FB08D608B2088E086AE3
:101482000846082307FF07DC07B9079607730751C9
:10149200072F070D06EC06CA06AA06890669064941
:1014A200062A060A05EC05CD05B005920575055814
:1014B200053C0520050504EA04CF04B5049C04821A
:1014C2000469045104390422040B03F403DE03C843
:1014D20003B2039D038903750361034D033B032894
:1014E2000316030402F202E102D102C002B002A01A
:1014F200029102820273026502570249023C022FE4
:1015020002220216020901FD01F201E601DB01D00D
:1015120001C601BB01B101A7019D0194018B0182AA
:1015220001790170016801600158015001480141CF
:1015320001390132012B0125011E01180111010B94
:10154200010500FF00FA0FA60FA00F990F920F8B53
:101552000F840F7C0F740F6B0F620F580F4E0F43E7
:101562000F380F2C0F1F0F120F050EF70EE80ED8B3
:101572000EC80EB70EA50E930E800E6C0E580E42BC
:101582000E2C0E150DFD0DE40DCB0DB10D950D7943
:101592000D5D0D3F0D200D010CE10CC00C9E0C7C6D
:1015A2000C590C350C100BEA0BC40B9E0B760B4F2F
:1015B2000B260AFD0AD40AAA0A800A550A2A09FF3A
:1015C20009D409A8097C0950092508F908CD08A100
:1015D2000875084A081E07F307C8079D07730749DD
:1015E200072006F706CE06A6067E06570630060A2E
:1015F20005E405BF059B057705540532051004EF88
:1016020004CE04AE048F047104530435041903FD9F
:1016120003E203C703AD0394037B0363034B033469
:10162200031E030802F302DE02CA02B602A30291FB
:10163200027F026D025C024C023C022C021D020E71
:10164200020001F201E401D701CA01BE01B101A603
:10165200019A018F0185017A01700166015D0153D2
:10166200014A014101390131012901210119011206
:10167200010B010400FD00F700F000EA00E400DEC7
:1016820000D900D300CE00C900C400BF00BA00B523
:1016920000B100AD00A800A400A0009C0099009534
:1016A2000091008E008A008700840081007E007B0A
:1016B20000001D0101010500020A0A5A0B000F0D6C
:1016C20000FA0E00020F013210009611006412019E
:1016D200321314FA14010215000217010A18010A42
:1016E200190A281A010A1B010A1C0A2823011E24AE
:1016F2000A642C50782D003C2E05462F001E300027
:1017020064325078330000343CFA350164360164A7
:10171200370150380A643B00013C00643E003C4102
:10172200145042005A430AC8440A3245007847011D
:1017320023480202500808510A9652143253000BF1
:10174200540A965601015705465C14325F006464E0
:081752000211650002FAFAFA27
:10004900750B00750A00AE0AAF0BAC08AD09EDC31C
:100059009FEC9E401674FF12184C75CF01780B74F3
:100069000126F6500418E436F650DB2290002BE006
:10007900B4AA0D900756E0B43C06E52A4529700359
:1000890002017B900029E4F0A3F075F809AE29AFCD
:100099002A74078E048F05FF121897ED4C700674A9
:1000A9003A900756F07E017F08E56F14121889907F
:1000B9000027EEF0A3EFF0900029E0FEA3E0FF7423
:1000C9000CD39F74019E5003020176A2F9B3500329
:1000D900020173EF4E700375A382900029E0FEA31D
:1000E900E0FF74016F4E700375A300900029E0FED4
:1000F900A3E0FF74026F4E700BE52A75F002A4FDB0
:10010900ACF08DA3900029E0FEA3E0FF74036F4ECD
:10011900700375A300900029E0FEA3E0FF7403BEFD
:1001290000039F5017900027E0FCA3E0FDED2FFF8F
:10013900EC3EFE9000521218A3E0F5A3900029E0CE
:10014900FEA3E0FFEFB40B09EEB401057414121815
:100159004C900029E0FEA3E0FFEFB40B07EEB401D9
:100169000375F80D90002912001E0200C090002BA3
:10017900E4F022752C00752B0075F8097E017F08C3
:10018900AC29AD2A1DBDFF011C12002E900021EEE5
:10019900F0A3EFF0AE2BAF2C7411D39F74019E50D6
:1001A9000302027CA2F9B35003020279E52C452B24
:1001B900700375A3D2AE2BAF2C74016F4E7003750B
:1001C900A300AE2BAF2C74026F4E700BE52A75F0AD
:1001D90002A4FDACF08DA3AE2BAF2C74036F4E704F
:1001E9000375A300AE2BAF2C74046F4E700375A377
:1001F90000AE2BAF2C74056F4E700375A300AE2BA8
:10020900AF2C74066F4E700375A300AE2BAF2C7420
:10021900076F4E700375A300AE2BAF2C74086F4E99
:10022900700375A300AE2BAF2C7408BE00039F505A
:100239001A900021E0FCA3E0FDED2FFFEC3EFE90BB
:10024900004D1218A3E5A3F075A300AE2BAF2CEF58
:10025900B41009EEB40105741412184CAE2BAF2C6E
:10026900EFB41007EEB4010375F80D782B1218CA14
:1002790002019D22C204C205C206C20722752C00D2
:10028900752B0075F809AE2BAF2C7417BE0004D37B
:100299009F500302035CA2F9B35003020359E52CF2
:1002A900452B700375A3D2AE2BAF2C74016F4E7022
:1002B9000375A300AE2BAF2C74026F4E700BE52AA9
:1002C90075F002A4FDACF08DA3AE2BAF2C74036FB7
:1002D9004E700375A300AE2BAF2C74046F4E7003E0
:1002E90075A300AE2BAF2C74056F4E700375A30078
:1002F900AE2BAF2C74066F4E700375A300AE2BAFF7
:100309002C74076F4E700375A300AE2BAF2C7408C5
:100319006F4E700375A300AE2BAF2C7408BE00039B
:100329009F500C90013C1218A3E5A3F075A300AEF1
:100339002BAF2C74166F4E7005741412184CAE2B1B
:10034900AF2C74166F4E700375F80D782B1218CAFE
:1003590002028F2290002BE0B4AB02800302041743
:10036900900029E4F0A3F075F809900029E0FEA3B4
:10037900E0FF7412BE0004D39F5003020417A2F9D0
:10038900B35003020414EF4E700375A38290002941
:10039900E0FEA3E0FF74016F4E700375A3009000A7
:1003A90029E0FEA3E0FF74026F4E700BE52A75F099
:1003B90002A4FDACF08DA3900029E0FEA3E0FF7438
:1003C900036F4E700375A300900029E0FEA3E0FFC0
:1003D9007403BE00039F50099000281218A3E0F58A
:1003E900A3900029E0FEA3E0FF74116F4E7005741D
:1003F9001412184C900029E0FEA3E0FF74116F4E0F
:10040900700375F80D90002912001E02037322C2B1
:10041900CF056D22900047E4936406600280FE7563
:10042900840175A70075FF8075EF0690002BE4F035
:1004390075C91075A70F75A1C775A70075D900757E
:10044900CE0C75A70F75F1FE75F2FF75F30775F4FC
:100459007875A4DA75A5FF75A60775AE0075AFFFA7
:1004690075D48175D5FF75D6FF75D7FF75A700754A
:10047900A20175A14775F80975D80075D90475DA0F
:100489000975DB0975E60875BC0175BE0475BD6C97
:1004990075BE0775BDA075BE0875BD0175BC007533
:1004A900BB1875BC2075BA0875E88075D11375A796
:1004B9000F75E10575E20075C74075B500C293C2B5
:1004C90094C291C292C287C290E5B554EFF5B5E5E1
:1004D900B554DFF5B5C296C295C2A0C297C2A2C2F1
:1004E900A1E5B554BFF5B5E5B5547FF5B5E5B55406
:1004F900FBF5B5759700759780740A12184C7597B6
:10050900C0E5975420700280F8758F0275A700D254
:10051900AF75980075A90C75A70F75AB4375ADFB41
:1005290075AC1E75A700758922758E04758C0075CA
:100539008A00C2A9D28CD2ADC2CFD2CA75D94475AC
:100549003E00753D00753A00753900754D00754ED0
:1005590000C29974C8F509750800120049756E0141
:10056900E56ED39407501B856E2A75290012017C0C
:100579007464F509750800120049786E740126F64D
:1005890050DE752A64752900120286752AC87529F4
:1005990000900145E0900008F0900146E0900009C4
:1005A900F0900147E090000AF0752A66752900125B
:1005B9000286752AC8752900740A90006EF0740ABB
:1005C900900071F0740A9000A7F07406900000F092
:1005D9007400900001F0900145E0900002F074036E
:1005E900900003F07405900004F07400900005F089
:1005F9007400900006F07400900007F0900146E046
:1006090090000BF0740090000CF0740090000DF055
:10061900740190000EF0740090000FF074FF9000C8
:1006290010F07400900063F090008AE0C3943C508D
:1006390006743C90008AF09000A7E0C3940A500623
:10064900740A9000A7F09000A9E0C3940A500674B8
:100659000A9000A9F012027D7559007527197528AD
:100669006490001174FFF0A374DCF0753E00753DD1
:1006790000756B00753800753700C2087570007514
:100689006100C20D75721E743A900756F074FD90A0
:100699000757F0C219757400900047E4F0754600D9
:1006A900754500900044E4F0A3F0900062E075F015
:1006B90032A4FFAEF08E418F4290001BE4F0A3F00C
:1006C90074FA90003DF0C21CC221A2B6B39200A2F6
:1006D900B3B39201A2B5B39202A2B4B39203755116
:1006E90046755200753000752F00C21B755B007589
:1006F9006900755E00755D007562327563327564F7
:1007090000743C90003BF0743C90003CF07566002E
:1007190075670075680090001FE4F0A3F0756A0022
:10072900756501900081E0900042F8E4F0E8A3F0DB
:10073900D2B2D2A4D2B0D2B1D2A3D2A7D2A6D2A5D4
:10074900D2B7900058E0D394FE400674FE9000584A
:10075900F0900059E0D394FE400674FE900059F0E1
:1007690090005AE0D394FE4006740A90005AF09023
:100779000080E0D394FE400674FE900080F0900063
:1007890081E0D394FE400674FE900081F074FF90DE
:100799000096F090009CE0D394FE400674FE900011
:1007A9009CF074FF90009FF09000A1E0D394014069
:1007B9000674009000A1F09000A2E0D394FE4006D8
:1007C90074FE9000A2F074FF9000A4F09000B4E0D1
:1007D900D39464400674649000B4F074FF9000B739
:1007E900F09000B8E0D394FE400674FE9000B8F093
:1007F90074FF9000B9F074009000BEF0740090008E
:10080900BFF0744D90012DF0746590012EF0747253
:1008190090012FF07463900130F07475900131F0FC
:100829007472900132F07479900133F0743290014E
:1008390034F07420900135F07454900136F07465E9
:10084900900137F07473900138F07474900139F0A5
:10085900742090013AF0742090013BF074009001EB
:1008690042F07400900143F07400900144F0D29C6E
:10087900D2EC75CF01A298B35003020B07C298E5D9
:100889004E6003020922754E00E599B4FF03754DC8
:1008990001E599B4FE03754D02E599B4FD03754D63
:1008A90003E599B4FC03754D04E599B4FA03754D54
:1008B90005E599B4FB03754E01E599D394E5400725
:1008C900E599C394F040028016859977754E027EAA
:1008D900017F00E577C394E61218898E3B8F3C753A
:1008E9003E00753D00E599D394C74007E599C39447
:1008F900E64002801F859977754E0374E5C39577A5
:10090900F53C753B00AE3BAF3C90136612183B7843
:100919003D1218B8D299020B07E54EB401028003C3
:10092900020A6FAE3DAF3E9000561218A3E599F04A
:10093900783D1218CAAE3DAF3EEFB40106EEB407DA
:10094900028003020A6F900756E0B43C028003025A
:100959000A69C29C12027D9000F4E090002CF0908C
:100969000063E090002DF0900083E090002EF0905D
:1009790000ACE090002FF0900058E0900030F0902B
:10098900009EE0900031F09000BCE0900032F090C1
:100999000090E0900033F09000AEE0900034F090C9
:1009A90000DEE0900035F0752A6375290074AB907C
:1009B900002BF012035D90002BE4F07464F50975C7
:1009C90008001200499000467401F0743C900756E3
:1009D900F0900046E01475F007A4FFAEF08F6E7535
:1009E9006F01E56FD394075024E56F256EF52A75DD
:1009F900290074AA90002BF01200757464F509752A
:100A09000800120049786F740126F650D57599FBD4
:100A19007402900046F0743C900756F0900046E04E
:100A29001475F007A4FFAEF08F6E756F01E56FD3F3
:100A390094075024E56F256EF52A75290074AA904C
:100A4900002BF01200757464F5097508001200494D
:100A5900786F740126F650D5752AC8752900D29C7D
:100A6900754E00754D00E54EB4024CE53E453D70AE
:100A79000685993A753900AE3DAF3E74016F4E70E7
:100A89001BAC39AD3AAA3BAB3CED2BFBEC3AFA8AED
:100A9900068B079000561218A3E599F0783D1218B5
:100AA900CAAE3DAF3E74026F4E700C12027D85775F
:100AB90099754E00754D00E54EB40342AE3DAF3E0B
:100AC9009000561218A3E599F0783D1218CAAE3D68
:100AD900AF3EAC3BAD3C8F028E038C068D07901365
:100AE900A212183BE493F9740193FEEAD39EEB99A1
:100AF900400C12027D857799754E00754D00E54DC4
:100B09006006A299B3B34003020C68C299E54DB4DB
:100B1900011FAE3DAF3E9000001218A3E0F5997891
:100B29003D1218CAAE3DAF3E74116F4E7003754D3C
:100B390000E54DB40203856599E54DB4031DAE3D4D
:100B4900AF3E9000561218A3E0F599EFB40107EEF5
:100B5900B40703754D00783D1218CAE54DB4040277
:100B69008003020C47E53E453D7003853099AE3D53
:100B7900AF3E74016F4E7003855B99AE3DAF3E7415
:100B8900026F4E7003855E99AE3DAF3E74036F4EA2
:100B99007003856299AE3DAF3E74046F4E70038554
:100BA9006499AE3DAF3E74056F4E7003856699AE8C
:100BB9003DAF3E74066F4E7003856799AE3DAF3EFB
:100BC90074076F4E7003856899AE3DAF3E74086F28
:100BD9004E7006900020E0F599AE3DAF3E74096F66
:100BE9004E700690003DE0F599AE3DAF3E74096F39
:100BF9004E700590003DE4F0AE3DAF3E740A6F4E75
:100C09007003856999AE3DAF3E740B6F4E700385D5
:100C19006399AE3DAF3E740C6F4E7003856A99AE11
:100C29003DAF3E740D6F4E70037599FC783D1218F7
:100C3900CAAE3DAF3E740E6F4E7003754D00E54D63
:100C4900B4051CAE3DAF3E9016B21218A3E493F55D
:100C59009974A76F4E7003754D00783D1218CAE557
:100C69004EB4010302087BC2CA7E107F00E56D12F3
:100C79001889E5CD75F010A4FDACF0EF2DFDEE3C23
:100C8900FCE5CC75F01084FF7E00ED2FFFEC3EFEF5
:100C99008E278F28D2CAA2B6300001B35003020DA5
:100CA90044A2B6300001B35003020D44A2B6300489
:100CB90001B3407AE55A705CE5284527601674014E
:100CC90012187B901362E493FC740193FD12175A76
:100CD9008E2F8F30AE2FAF307428BE00039F501077
:100CE900E5612FFF50010E740112187B8E2F8F3092
:100CF9008530619000A7E0A82FB8000DD39530404A
:100D090008E53090003AF080099000A7E0149000BF
:100D19003AF08002155AC2CA75CD0075CC00756DBE
:100D290000752801752700D2CAA204B39200A20453
:100D3900B330B601B34004A204920090001112002E
:100D49001E900011E0FEA3E0FFEFB47006EEB417A9
:100D59000280030210BF900011E4F0A3F00552E5F0
:100D690052B40A48E5B554FEF5B5E5B554BFF5B535
:100D7900C2A2C2A0C296E5B554F7F5B5C293C29115
:100D8900C287E5B554EFF5B5E5B554FDF5B5E5B55B
:100D9900547FF5B5C2A1C297C295E5B554FBF5B527
:100DA900C294C292C290E5B554DFF5B5E552B414C8
:100DB90048E5B54401F5B5E5B54440F5B5D2A2D24B
:100DC900A0D296E5B54408F5B5D293D291D287E57C
:100DD900B54410F5B5E5B54402F5B5E5B5547FF56B
:100DE900B5C2A1C297C295E5B554FBF5B5C294C287
:100DF90092C290E5B554DFF5B5E552B41E48E5B5A4
:100E090054FEF5B5E5B554BFF5B5C2A2C2A0C29668
:100E1900E5B554F7F5B5C293C291C287E5B554EF6C
:100E2900F5B5E5B554FDF5B5E5B54480F5B5D2A1FF
:100E3900D297D295E5B54404F5B5D294D292D29021
:100E4900E5B54420F5B5E552B42848E5B554FEF5B5
:100E5900B5E5B554BFF5B5C2A2C2A0C296E5B55471
:100E6900F7F5B5C293C291C287E5B554EFF5B5E57B
:100E7900B554FDF5B5E5B5547FF5B5C2A1C297C224
:100E890095E5B554FBF5B5C294C292C290E5B55447
:100E9900DFF5B5E552B43248E5B54401F5B5E5B538
:100EA90054BFF5B5C2A2C2A0C296E5B554F7F5B5CF
:100EB900C293C291C287E5B554EFF5B5E5B54402D1
:100EC900F5B5E5B5547FF5B5C2A1C297C295E5B5AB
:100ED90054FBF5B5C294C292C290E5B554DFF5B59D
:100EE900E552B43C48E5B554FEF5B5E5B54440F5E1
:100EF900B5C2A2C2A0C296E5B554F7F5B5C293C270
:100F090091C287E5B54410F5B5E5B554FDF5B5E5EC
:100F1900B54480F5B5C2A1C297C295E5B554FBF5B4
:100F2900B5C294C292C290E5B54420F5B5E552B474
:100F39004648E5B554FEF5B5E5B554BFF5B5D2A2B9
:100F4900C2A0C296E5B554F7F5B5C293C291D2874E
:100F5900E5B554EFF5B5E5B554FDF5B5E5B5547FFF
:100F6900F5B5D2A1C297C295E5B554FBF5B5C294C2
:100F7900C292D290E5B554DFF5B5E552B45048E5D3
:100F8900B554FEF5B5E5B554BFF5B5C2A2D2A0C2B8
:100F990096E5B554F7F5B5C293D291C287E5B55434
:100FA900EFF5B5E5B554FDF5B5E5B5547FF5B5C231
:100FB900A1D297C295E5B554FBF5B5C294D292C2B8
:100FC90090E5B554DFF5B5E552B45A48E5B554FE98
:100FD900F5B5E5B554BFF5B5C2A2C2A0D296E5B53F
:100FE90054F7F5B5D293C291C287E5B554EFF5B57B
:100FF900E5B554FDF5B5E5B5547FF5B5C2A1C29780
:10100900D295E5B554FBF5B5D294C292C290E5B537
:1010190054DFF5B5E552B46448E5B554FEF5B5E5D8
:10102900B554BFF5B5C2A2C2A0C296E5B54408F54C
:10103900B5C293C291C287E5B554EFF5B5E5B5548C
:10104900FDF5B5E5B5547FF5B5C2A1C297C295E5E1
:10105900B54404F5B5C294C292C290E5B554DFF522
:10106900B5E552B46E48E5B554FEF5B5E5B554BFDE
:10107900F5B5C2A2C2A0C296E5B554F7F5B5C293BB
:10108900C291C287E5B554EFF5B5E5B554FDF5B59F
:10109900E5B5547FF5B5C2A1C297C295E5B554FB34
:1010A900F5B5C294C292C290E5B554DFF5B5E552E3
:1010B900B48C0375520AE552D3946E4054A2B640DB
:1010C90006E5B554FBF5B5A2B6B34006E5B544044B
:1010D900F5B5A2B34006E5B554DFF5B5A2B3B34003
:1010E90006E5B54420F5B5A2B54006E5B5547FF54A
:1010F900B5A2B5B34006E5B54480F5B5A2B440063E
:10110900E5B554BFF5B5A2B4B34006E5B54440F51D
:10111900B5E56BB40A03756B00E56BC3940A40032C
:1011290002132DA2EDB3500302132DC2EDE56B702E
:101139001E7E017F00E5BE121889E5BD2FFF500113
:101149000E8E318F32740412187B8F5B75BB18E5D4
:101159006BB401207E017F00E5BE121889E5BD2F21
:10116900FF50010E8E318F32740412187B8E5D8F01
:101179005E75BB19E56BB402237E017F00E5BE12E3
:101189001889E5BD2FFF50010E8E318F3274298EDB
:10119900048F05FF12185C8D6275BB13E56BB403F0
:1011A9001E7E017F00E5BE121889E5BD2FFF5001A3
:1011B9000E8E318F32740412187B8F6375BB17E55D
:1011C9006BB404727E017F00E5BE121889E5BD2F5C
:1011D900FF50010E8E318F3290003BE06019900074
:1011E9003BE0149013DE12186CE493FC740193FD38
:1011F900EDC39FEC9E4002800690003BE014F09006
:10120900003BE0C394B3501DAE31AF3290003BE0D8
:10121900049013DE12186CE493FC740193FDEFC380
:101229009DEE9C4002800690003BE004F090003B5C
:10123900E0F56475BB16E56BB405727E017F00E5C8
:10124900BE121889E5BD2FFF50010E8E318F3290E5
:10125900003CE0601990003CE01490154812186CAD
:10126900E493FC740193FDEDC39FEC9E400280065C
:1012790090003CE014F090003CE0C394B3501DAEE4
:1012890031AF3290003CE00490154812186CE49399
:10129900FC740193FDEFC39DEE9C40028006900013
:1012A9003CE004F090003CE0F56675BB1FE56BB4CB
:1012B90006287E017F00E5BE121889E5BD2FFF5083
:1012C900010E8E318F32740912188974E68E048FDB
:1012D90005FF12185C8D6875BB15E56BB4071E7E9A
:1012E900017F00E5BE121889E5BD2FFF50010E8E62
:1012F900318F32740412187B8F6775BB14E56BB498
:10130900081E7E017F00E5BE121889E5BD2FFF503A
:10131900010E8E318F32740412187B8F6975BB1AD6
:10132900056BD2ECAE27AF28EFD394DCEE94FF40E7
:1013390025755146755A02753000752F0075610083
:1013490090001FE4F0A3F075280075270075CD0003
:0913590075CC00756D0002087BE3
:0F186C0025E050020583258250020583F5822274
:10183B00EF2F500205832582F582E5833E2EF5833B
:01184B00227A
:0918B800E493F608740193F62292
:0818CA000806B6000218062210
:0D001E00A3E004F070061218AEE004F0221A
:0E187B00048007C3CE13CECF13CFD5E0F622E4
:10175A00BC000FBE0008ED8FF084FFADF022E4FE5E
:10176A00FF22BE000DEF60FE54F0606F20E7030217
:10177A001810EAC0E0EBC0E078017A0075F001EEDB
:10178A0020E710EF25E0FFEE33FE0AC5F023C5F08F
:10179A0030E7F0EA5407F9096A7A007B0060010829
:1017AA00C3EC9E40167004ED9F4010ED9FFDEC9E29
:1017BA00FCE5F0CA4ACA03F5F08005E5F003F5F046
:1017CA00C3EE13FEEF13FFD9D77908CACBCAD8D014
:1017DA00EAFEEBFFD0E0FBD0E0FA22EC8FF084FCCB
:1017EA00ED54F045F0C48FF084FEEDC454F045F09A
:1017FA00C48FF084FDEEC4FE54F02DFFEE540F3C6E
:10180A00FEADF07C0022790078008FF0EC7E082093
:10181A00E70DC3CD33CD33C933C9C833C8DEF0842D
:10182A0049F9E5F08FF0BE00E6FD7C00E9FFE8FE2D
:01183A00228B
:0E188900F88FF0A4FFE5F0CE88F0A42EFE222A
:10002E00EF8DF0A4F9A8F0EF8CF0A428F8EE8DF087
:06003E00A428FEE9FF22E8
:10184C00600D782B021856007830D8FED5E0F822BF
:10185C00EEC0E07E0012175AEFFDEEFCD0E0FE2247
:0C189700EEC0E07E0012175AD0E0FE22E6
:03002B00020003CD
:030000000218C122
:0918C10075817D75D00002041D43
:1018A300E5822FF582E5833EF583220582D5820208
:0518B3001583158222DF
:10000300C0E0C0F0C083C082C0D075D00012041815
:0B001300D0D0D082D083D0F0D0E032FB
:00000001FF
